:03000000020C00EF
:03000300021A03DB
:03000B00021A06D0
:03001300021A09C5
:03001B00021A0CBA
:03002300021A0FAF
:03002B00021A12A4
:03003300021A1599
:03003B00021A188E
:03004300021A1B83
:03004B00021A1E78
:03005300021A216D
:03005B00021A2462
:03006300021A2757
:03006B00021A2A4C
:03007300021A2D41
:03007B00021A3036
:03008300021A332B
:03008B00021A3620
:03009300021A3915
:03009B00021A3C0A
:0300A300021A3FFF
:100C0000787FE4F6D8FD9000007F007E20E4F0A31A
:0A0C1000DFFCDEFA758120020C55AE
:101A3C0006012C034D056E078F09A70B0000000053
:101A4C0000000032006400C8012C015E019001C24C
:101A5C0001FC022E0261029402C702FA032C035FFE
:101A6C00039203C503F8042A045D049004C304F62E
:101A7C000528055B058E05C105F406260659068C5E
:101A8C0006BF06F207240757078A07BD07F008228E
:101A9C000855088808BB08EE09210953098609B9BD
:101AAC0009EC0A1F0A510A840AB70AEA0B1D0B4FEC
:101ABC000B820BB50BE80C1B0C4D0C800CB30CE61D
:101ACC000D190D4B0D7E0DB10DE40E170E490E7C4C
:101ADC000EAF0EE20F150F470F7A0FAD0FE010137C
:101AEC001045107810AB10DE11111144117611A9AC
:101AFC0011DC120F1242127412A712DA130D1340DA
:101B0C00137213A513D8140B143E147014A314D60B
:101B1C001509153C156E15A115D41607163A166C39
:101B2C00169F16D217051738176A179D17D018036A
:101B3C0018361868189B18CE190119341967199999
:101B4C0019CC19FF1A321A651A971ACA1AFD1B30CA
:101B5C001B631B951BC81BFB1C2E1C611C931CC6FA
:101B6C001CF91D2C1D5F1D911DC41DF71E2A1E5D29
:101B7C001E8F1EC21EF51F281F5B1F8D1FC01FF35B
:101B8C0020262059208B20BE20F121242157218989
:101B9C0021BC21EF22222255228822BA22ED2320B9
:101BAC002353238623B823EB241E2451248424B6E8
:101BBC0024E9251C254F258225B425E7261A264D18
:101BCC00268026B226E52718274B277E27B027E349
:101BDC0028162849287C28AE28E129142947297A77
:101BEC0029AC29DF2A122A452A782AAB2ADD2B10A8
:101BFC002B432B762BA92BDB2C0E2C412C742CA7D6
:101C0C002CD92D0C2D3F2D722DA52DD72E0A2E3D06
:101C1C002E702EA32ED52F082F3B2F6E2FA12FD336
:101C2C0030063039306C309F30D131043137316A65
:101C3C00319D31CF320232353268329B32CE330095
:101C4C0033333366339933CC33FE343134643497C5
:101C5C0034CA34FC352F3562359535C835FA362DF6
:101C6C003660369336C636F8372B375E379137C425
:101C7C0037F63829385C388F38C238F43927395A56
:101C8C00398D39C039F23A253A583A8B3ABE3AF086
:101C9C003B233B563B893BBC3BEF3C213C543C87B4
:101CAC003CBA3CED3D1F3D523D853DB83DEB3E1DE4
:101CBC003E503E833EB63EE93F1B3F4E3F813FB414
:101CCC003FE74019404C407F40B240E54117414A44
:101CDC00417D41B041E342154248427B42AE42E174
:101CEC0043134346437943AC43DF441244444477A3
:101CFC0044AA44DD45104542457545A845DB460ED2
:101D0C004640467346A646D9470C473E477147A402
:101D1C0047D7480A483C486F48A248D54908493A31
:101D2C00496D49A049D34A064A384A6B4A9E4AD162
:101D3C004B044B364B694B9C4BCF4C024C354C6790
:101D4C004C9A4CCD4D004D334D654D984DCB4DFEC1
:101D5C004E314E634E964EC94EFC4F2F4F614F94F1
:101D6C004FC74FFA502D505F509250C550F8512B21
:101D7C00515D519051C351F65229525B528E52C152
:101D8C0052F453275359538C53BF53F25425545781
:101D9C00548A54BD54F055235556558855BB55EEB1
:101DAC0056215654568656B956EC571F57525784DF
:101DBC0057B757EA581D5850588258B558E8591B10
:101DCC00594E598059B359E65A195A4C5A7E5AB140
:101DDC005AE45B175B4A5B7C5BAF5BE25C155C486F
:101DEC005C7A5CAD5CE05D135D465D795DAB5DDEA0
:101DFC005E115E445E775EA95EDC5F0F5F425F75CD
:101E0C005FA75FDA600D6040607360A560D8610BFE
:101E1C00613E617161A361D66209623C626F62A12D
:101E2C0062D46307633A636D639F63D2640564385D
:101E3C00646B649D64D0650365366569659B65A7B5
:101E4C0065B265BD65C865D365DE65E965F465FF9A
:101E5C00660A66156620662B66366641664C6657C2
:101E6C006662666D66786683668E669966A466AFF2
:101E7C0066BA66C566D066DB66E666F166FC670820
:101E8C006713671E67296734673F674A6755676042
:101E9C00676B67766781678C679767A267AD67B872
:101EAC0067C367CE67D967E467EF67FA68056810A0
:101EBC00681B68266831683C68476852685D6868CA
:101ECC006874687F688A689568A068AB68B668C1F2
:101EDC0068CC68D768E268ED68F86903690E69191F
:101EEC006924692F693A69456950695B696669714A
:101EFC00697C69876992699D69A869B369BE69C97A
:101F0C0069D569E069EB69F66A016A0C6A176A229D
:101F1C006A2D6A386A436A4E6A596A646A6F6A7AC9
:101F2C006A856A906A9B6AA66AB16ABC6AC76AD2F9
:101F3C006ADD6AE86AF36AFE6B096B146B1F6B2A25
:101F4C006B356B416B4C6B576B626B6D6B786B834A
:101F5C006B8E6B996BA46BAF6BBA6BC56BD06BDB79
:101F6C006BE66BF16BFC6C076C126C1D6C286C33A4
:101F7C006C3E6C496C546C5F6C6A6C756C806C8BD1
:101F8C006C966CA26CAD6CB86CC36CCE6CD96CE4FA
:101F9C006CEF6CFA6D056D106D1B6D266D316D3C23
:101FAC006D476D526D5D6D686D736D7E6D896D9451
:101FBC006D9F6DAA6DB56DC06DCB6DD66DE16DEC81
:101FCC006DF76E026E0E6E196E246E2F6E3A6E45A4
:101FDC006E506E5B6E666E716E7C6E876E926E9DD1
:101FEC006EA86EB36EBE6EC96ED46EDF6EEA6EF501
:101FFC006F006F0B6F166F216F2C6F376F426F4D29
:10200C006F586F636F6E6F7A6F856F906F9B6FA653
:10201C006FB16FBC6FC76FD26FDD6FE86FF36FFE80
:10202C0070097014701F702A70357040704B7056A8
:10203C007061706C70777082708D709870A370AED8
:10204C0070B970C470CF70DB70E670F170FC710702
:10205C007112711D71287133713E71497154715F28
:10206C00716A71757180718B719671A171AC71B758
:10207C0071C271CD71D871E371EE71F97204720F86
:10208C00721A72257230723B72477252725D7268AC
:10209C007273727E72897294729F72AA72B572C0D8
:1020AC0072CB72D672E172EC72F77302730D731805
:1020BC007323732E73397344734F735A7365737030
:1020CC00737B73867391739C73A873B373BE73C95C
:1020DC0073D473DF73EA73F57400740B7416742184
:1020EC00742C74377442744D74587463746E7479B0
:1020FC007484748F749A74A574B074BB74C674D1E0
:10210C0074DC74E774F274FD75087514751F752A08
:10211C0075357540754B75567561756C757775822F
:10212C00758D759875A375AE75B975C475CF75DA5F
:10213C0075E575F075FB76067611761C762776328A
:10214C00763D76487653765E766976757680768BB4
:10215C00769676A176AC76B776C276CD76D876E3DF
:10216C0076EE76F97704770F771A77257730773B09
:10217C0077467751775C77677772777D7788779337
:10218C00779E77A977B477BF77CA77D577E177EC65
:10219C0077F77802780D78187823782E7839784488
:1021AC00784F785A78657870787B78867891789CB7
:1021BC0078A778B278BD78C878D378DE78E978F4E7
:1021CC0078FF790A79157920792B79367941794D0F
:1021DC0079587963796E79797984798F799A79A537
:1021EC0079B079BB79C679D179DC79E779F279FD67
:1021FC007A087A137A1E7A297A347A3F7A4A7A558F
:10220C007A607A6B7A767A817A8C7A977AA27AAEBD
:10221C007AB97AC47ACF7ADA7AE57AF07AFB7B06E5
:10222C007B117B1C7B277B327B3D7B487B537B5E0E
:10223C007B697B747B7F7B8A7B957BA07BAB7BB63E
:10224C007BC17BCC7BD77BE27BED7BF87C037C0E6C
:10225C007C1A7C257C307C3B7C467C517C5C7C678E
:10226C007C727C7D7C887C937C9E7CA97CB47CBFBE
:10227C007CCA7CD57CE07CEB7CF67D017D0C7D17EB
:10228C007D227D2D7D387D437D4E7D597D647D6F16
:10229C007D7B7D867D917D9C7DA77DB27DBD7DC83E
:1022AC007DD37DDE7DE97DF47DFF7E0A7E157E206B
:1022BC007E2B7E367E417E4C7E577E627E6D7E7896
:1022CC007E837E8E7E997EA47EAF7EBA7EC57ED0C6
:1022DC007EDB7EE77EF27EFD7F087F137F1E7F29EB
:1022EC007F347F3F7F4A7F557F607F6B7F767F8116
:1022FC007F8C7F977FA27FAD7FB87FC37FCE7FD946
:10230C007FE47FEF7FFA80058010801B8026803170
:10231C00803C80488053805E80698074807F808A96
:10232C00809580A080AB80B680C180CC80D780E2C5
:10233C0080ED80F88103810E81198124812F813AEF
:10234C0081458150815B81668171817C818781921D
:10235C00819D81A881B481BF81CA81D581E081EB47
:10236C0081F68201820C82178222822D823882436E
:10237C00824E82598264826F827A82858290829B9D
:10238C0082A682B182BC82C782D282DD82E882F3CD
:10239C0082FE830983148320832B83368341834CF1
:1023AC0083578362836D83788383838E839983A41D
:1023BC0083AF83BA83C583D083DB83E683F183FC4D
:1023CC0084078412841D84288433843E8449845475
:1023DC00845F846A84758481848C849784A284ADA0
:1023EC0084B884C384CE84D984E484EF84FA8505CC
:1023FC008510851B85268531853C85478552855DF5
:10240C0085688573857E85898594859F85AA85B524
:10241C0085C085CB85D685E185ED85F88603860E4E
:10242C0086198624862F863A86458650865B866674
:10243C008671867C86878692869D86A886B386BEA4
:10244C0086C986D486DF86EA86F58700870B8716D1
:10245C008721872C87378742874E87598764876FF8
:10246C00877A87858790879B87A687B187BC87C724
:10247C0087D287DD87E887F387FE88098814881F51
:10248C00882A88358840884B88568861886C88777C
:10249C008882888D889888A388AE88BA88C588D0A9
:1024AC0088DB88E688F188FC89078912891D8928D0
:1024BC008933893E89498954895F896A89758980FC
:1024CC00898B899689A189AC89B789C289CD89D82C
:1024DC0089E389EE89F98A048A0F8A1B8A268A3154
:1024EC008A3C8A478A528A5D8A688A738A7E8A897C
:1024FC008A948A9F8AAA8AB58AC08ACB8AD68AE1AC
:10250C008AEC8AF78B028B0D8B188B238B2E8B39D5
:10251C008B448B4F8B5A8B658B708B7B8B878B9201
:10252C008B9D8BA88BB38BBE8BC98BD48BDF8BEA2B
:10253C008BF58C008C0B8C168C218C2C8C378C4254
:10254C008C4D8C588C638C6E8C798C848C8F8C9A83
:10255C008CA58CB08CBB8CC68CD18CDC8CE78CF3B2
:10256C008CFE8D098D148D1F8D2A8D358D408D4BD4
:10257C008D568D618D6C8D778D828D8D8D988DA303
:10258C008DAE8DB98DC48DCF8DDA8DE58DF08DFB33
:10259C008E068E118E1C8E278E328E3D8E488E545A
:1025AC008E5F8E6A8E758E808E8B8E968EA18EAC83
:1025BC008EB78EC28ECD8ED88EE38EEE8EF98F04B2
:1025CC008F0F8F1A8F258F308F3B8F468F518F5CDB
:1025DC008F678F728F7D8F888F938F9E8FA98FB40B
:1025EC008FC08FCB8FD68FE18FEC8FF79002900D31
:1025FC0090189023902E90399044904F905A90655B
:10260C009070907B90869091909C90A790B290BD8A
:10261C0090C890D390DE90E990F490FF910A9115B8
:10262C009121912C91379142914D91589163916EDA
:10263C0091799184918F919A91A591B091BB91C60A
:10264C0091D191DC91E791F291FD92089213921E37
:10265C0092299234923F924A92559260926B927662
:10266C009281928D929892A392AE92B992C492CF8B
:10267C0092DA92E592F092FB93069311931C9327B6
:10268C009332933D93489353935E93699374937FE2
:10269C00938A939593A093AB93B693C193CC93D712
:1026AC0093E293EE93F99404940F941A9425943036
:1026BC00943B94469451945C94679472947D948862
:1026CC009493949E94A994B494BF94CA94D594E092
:1026DC0094EB94F69501950C95179522952D9538BC
:1026EC009543954E955A95659570957B95869591E4
:1026FC00959C95A795B295BD95C895D395DE95E912
:10270C0095F495FF960A96159620962B963696413B
:10271C00964C96579662966D96789683968E969969
:10272C0096A496AF96BA96C696D196DC96E796F294
:10273C0096FD97089713971E97299734973F974ABA
:10274C0097559760976B97769781978C979797A2E9
:10275C0097AD97B897C397CE97D997E497EF97FA19
:10276C0098059810981B98279832983D984898533C
:10277C00985E98699874987F988A989598A098AB69
:10278C0098B698C198CC98D798E298ED98F8990398
:10279C00990E99199924992F993A99459950995BC1
:1027AC0099669971997C99879993999E99A999B4ED
:1027BC0099BF99CA99D599E099EB99F69A019A0C17
:1027CC009A179A229A2D9A389A439A4E9A599A6441
:1027DC009A6F9A7A9A859A909A9B9AA69AB19ABC71
:1027EC009AC79AD29ADD9AE89AF49AFF9B0A9B159B
:1027FC009B209B2B9B369B419B4C9B579B629B6DC1
:10280C009B789B839B8E9B999BA49BAF9BBA9BC5F0
:10281C009BD09BDB9BE69BF19BFC9C079C129C1D1D
:10282C009C289C339C3E9C499C549C609C6B9C7645
:10283C009C819C8C9C979CA29CAD9CB89CC39CCE70
:10284C009CD99CE49CEF9CFA9D059D109D1B9D269C
:10285C009D319D3C9D479D529D5D9D689D739D7EC8
:10286C009D899D949D9F9DAA9DB59DC19DCC9DD7F5
:10287C009DE29DED9DF89E039E0E9E199E249E2F1B
:10288C009E3A9E459E509E5B9E669E719E7C9E8748
:10289C009E929E9D9EA89EB39EBE9EC99ED49EDF78
:1028AC009EEA9EF59F009F0B9F169F219F2D9F38A0
:1028BC009F439F4E9F599F649F6F9F7A9F859F90C8
:1028CC009F9B9FA69FB19FBC9FC79FD29FDD9FE8F8
:1028DC009FF39FFEA009A014A01FA02AA035A04022
:1028EC00A04BA056A061A06CA077A082A08DA0994F
:1028FC00A0A4A0AFA0BAA0C5A0D0A0DBA0E6A0F178
:10290C00A0FCA107A112A11DA128A133A13EA149A0
:10291C00A154A15FA16AA175A180A18BA196A1A1CF
:10292C00A1ACA1B7A1C2A1CDA1D8A1E3A1EEA1FAFE
:10293C00A205A210A21BA226A231A23CA247A2521F
:10294C00A25DA268A273A27EA289A294A29FA2AA4F
:10295C00A2B5A2C0A2CBA2D6A2E1A2ECA2F7A3027E
:10296C00A30DA318A323A32EA339A344A34FA35AA7
:10297C00A366A371A37CA387A392A39DA3A8A3B3CF
:10298C00A3BEA3C9A3D4A3DFA3EAA3F5A400A40BFD
:10299C00A416A421A42CA437A442A44DA458A46327
:1029AC00A46EA479A484A48FA49AA4A5A4B0A4BB57
:1029BC00A4C7A4D2A4DDA4E8A4F3A4FEA509A5147D
:1029CC00A51FA52AA535A540A54BA556A561A56CA7
:1029DC00A577A582A58DA598A5A3A5AEA5B9A5C4D7
:1029EC00A5CFA5DAA5E5A5F0A5FBA606A611A61C04
:1029FC00A627A633A63EA649A654A65FA66AA67528
:102A0C00A680A68BA696A6A1A6ACA6B7A6C2A6CD56
:102A1C00A6D8A6E3A6EEA6F9A704A70FA71AA72582
:102A2C00A730A73BA746A751A75CA767A772A77DAE
:102A3C00A788A794A79FA7AAA7B5A7C0A7CBA7D6D7
:102A4C00A7E1A7ECA7F7A802A80DA818A823A82E01
:102A5C00A839A844A84FA85AA865A870A87BA8862E
:102A6C00A891A89CA8A7A8B2A8BDA8C8A8D3A8DE5E
:102A7C00A8E9A8F4A900A90BA916A921A92CA93782
:102A8C00A942A94DA958A963A96EA979A984A98FAE
:102A9C00A99AA9A5A9B0A9BBA9C6A9D1A9DCA9E7DE
:102AAC00A9F2A9FDAA08AA13AA1EAA29AA34AA3F08
:102ABC00AA4AAA55AA60AA6CAA77AA82AA8DAA9831
:102ACC00AAA3AAAEAAB9AAC4AACFAADAAAE5AAF05E
:102ADC00AAFBAB06AB11AB1CAB27AB32AB3DAB4887
:102AEC00AB53AB5EAB69AB74AB7FAB8AAB95ABA0B6
:102AFC00ABABABB6ABC1ABCDABD8ABE3ABEEABF9E1
:102B0C00AC04AC0FAC1AAC25AC30AC3BAC46AC5105
:102B1C00AC5CAC67AC72AC7DAC88AC93AC9EACA935
:102B2C00ACB4ACBFACCAACD5ACE0ACEBACF6AD0164
:102B3C00AD0CAD17AD22AD2DAD39AD44AD4FAD5A89
:102B4C00AD65AD70AD7BAD86AD91AD9CADA7ADB2B5
:102B5C00ADBDADC8ADD3ADDEADE9ADF4ADFFAE0AE4
:102B6C00AE15AE20AE2BAE36AE41AE4CAE57AE620D
:102B7C00AE6DAE78AE83AE8EAE9AAEA5AEB0AEBB39
:102B8C00AEC6AED1AEDCAEE7AEF2AEFDAF08AF1363
:102B9C00AF1EAF29AF34AF3FAF4AAF55AF60AF6B8D
:102BAC00AF76AF81AF8CAF97AFA2AFADAFB8AFC3BD
:102BBC00AFCEAFD9AFE4AFEFAFFAB006B011B01CE7
:102BCC00B027B032B03DB048B053B05EB069B0740D
:102BDC00B07FB08AB095B0A0B0ABB0B6B0C1B0CC3D
:102BEC00B0D7B0E2B0EDB0F8B103B10EB119B12469
:102BFC00B12FB13AB145B150B15BB167B172B17D92
:102C0C00B188B193B19EB1A9B1B4B1BFB1CAB1D5BC
:102C1C00B1E0B1EBB1F6B201B20CB217B222B22DE7
:102C2C00B238B243B24EB259B264B26FB27AB28514
:102C3C00B290B29BB2A6B2B1B2BCB2C7B2D3B2DE42
:102C4C00B2E9B2F4B2FFB30AB315B320B32BB33667
:102C5C00B341B34CB357B362B36DB378B383B38E94
:102C6C00B399B3A4B3AFB3BAB3C5B3D0B3DBB3E6C4
:102C7C00B3F1B3FCB407B412B41DB428B433B43FED
:102C8C00B44AB455B460B46BB476B481B48CB49714
:102C9C00B4A2B4ADB4B8B4C3B4CEB4D9B4E4B4EF44
:102CAC00B4FAB505B510B51BB526B531B53CB5476D
:102CBC00B552B55DB568B573B57EB589B594B5A09B
:102CCC00B5ABB5B6B5C1B5CCB5D7B5E2B5EDB5F8C4
:102CDC00B603B60EB619B624B62FB63AB645B650EC
:102CEC00B65BB666B671B67CB687B692B69DB6A81C
:102CFC00B6B3B6BEB6C9B6D4B6DFB6EAB6F5B7004B
:102D0C00B70CB717B722B72DB738B743B74EB7596B
:102D1C00B764B76FB77AB785B790B79BB7A6B7B19B
:102D2C00B7BCB7C7B7D2B7DDB7E8B7F3B7FEB809CA
:102D3C00B814B81FB82AB835B840B84BB856B861F3
:102D4C00B86DB878B883B88EB899B8A4B8AFB8BA1B
:102D5C00B8C5B8D0B8DBB8E6B8F1B8FCB907B91249
:102D6C00B91DB928B933B93EB949B954B95FB96A73
:102D7C00B975B980B98BB996B9A1B9ACB9B7B9C2A3
:102D8C00B9CDB9D9B9E4B9EFB9FABA05BA10BA1BC9
:102D9C00BA26BA31BA3CBA47BA52BA5DBA68BA73F3
:102DAC00BA7EBA89BA94BA9FBAAABAB5BAC0BACB23
:102DBC00BAD6BAE1BAECBAF7BB02BB0DBB18BB234F
:102DCC00BB2EBB3ABB45BB50BB5BBB66BB71BB7C74
:102DDC00BB87BB92BB9DBBA8BBB3BBBEBBC9BBD4A3
:102DEC00BBDFBBEABBF5BC00BC0BBC16BC21BC2CCE
:102DFC00BC37BC42BC4DBC58BC63BC6EBC79BC84FB
:102E0C00BC8FBC9ABCA6BCB1BCBCBCC7BCD2BCDD24
:102E1C00BCE8BCF3BCFEBD09BD14BD1FBD2ABD354D
:102E2C00BD40BD4BBD56BD61BD6CBD77BD82BD8D7A
:102E3C00BD98BDA3BDAEBDB9BDC4BDCFBDDABDE5AA
:102E4C00BDF0BDFBBE06BE12BE1DBE28BE33BE3ECF
:102E5C00BE49BE54BE5FBE6ABE75BE80BE8BBE96FA
:102E6C00BEA1BEACBEB7BEC2BECDBED8BEE3BEEE2A
:102E7C00BEF9BF04BF0FBF1ABF25BF30BF3BBF4653
:102E8C00BF51BF5CBF67BF73BF7EBF89BF94BF9F7D
:102E9C00BFAABFB5BFC0BFCBBFD6BFE1BFECBFF7AA
:102EAC00C002C00DC018C023C02EC039C044C04FD2
:102EBC00C05AC065C070C07BC086C091C09CC0A702
:102ECC00C0B2C0BDC0C8C0D3C0DFC0EAC0F5C1002D
:102EDC00C10BC116C121C12CC137C142C14DC15852
:102EEC00C163C16EC179C184C18FC19AC1A5C1B082
:102EFC00C1BBC1C6C1D1C1DCC1E7C1F2C1FDC208B1
:102F0C00C213C21EC229C234C240C24BC256C261D5
:102F1C00C26CC277C282C28DC298C2A3C2AEC2B901
:102F2C00C2C4C2CFC2DAC2E5C2F0C2FBC306C3112F
:102F3C00C31CC327C332C33DC348C353C35EC36959
:102F4C00C374C37FC38AC395C3A0C3ACC3B7C3C286
:102F5C00C3CDC3D8C3E3C3EEC3F9C404C40FC41AAE
:102F6C00C425C430C43BC446C451C45CC467C472D9
:102F7C00C47DC488C493C49EC4A9C4B4C4BFC4CA09
:102F8C00C4D5C4E0C4EBC4F6C501C50DC518C52332
:102F9C00C52EC539C544C54FC55AC565C570C57B59
:102FAC00C586C591C59CC5A7C5B2C5BDC5C8C5D389
:102FBC00C5DEC5E9C5F4C5FFC60AC615C620C62BB5
:102FCC00C636C641C64CC657C662C66DC679C684DF
:102FDC00C68FC69AC6A5C6B0C6BBC6C6C6D1C6DC09
:102FEC00C6E7C6F2C6FDC708C713C71EC729C73434
:102FFC00C73FC74AC755C760C76BC776C781C78C61
:10300C00C797C7A2C7ADC7B8C7C3C7CEC7D9C7E58F
:10301C00C7F0C7FBC806C811C81CC827C832C83DB2
:10302C00C848C853C85EC869C874C87FC88AC895E0
:10303C00C8A0C8ABC8B6C8C1C8CCC8D7C8E2C8ED10
:10304C00C8F8C903C90EC919C924C92FC93AC94638
:10305C00C951C95CC967C972C97DC988C993C99E60
:10306C00C9A9C9B4C9BFC9CAC9D5C9E0C9EBC9F690
:10307C00CA01CA0CCA17CA22CA2DCA38CA43CA4EB8
:10308C00CA59CA64CA6FCA7ACA85CA90CA9BCAA6E8
:10309C00CAB2CABDCAC8CAD3CADECAE9CAF4CAFF10
:1030AC00CB0ACB15CB20CB2BCB36CB41CB4CCB5738
:1030BC00CB62CB6DCB78CB83CB8ECB99CBA4CBAF68
:1030CC00CBBACBC5CBD0CBDBCBE6CBF1CBFCCC0797
:1030DC00CC13CC1ECC29CC34CC3FCC4ACC55CC60B8
:1030EC00CC6BCC76CC81CC8CCC97CCA2CCADCCB8E8
:1030FC00CCC3CCCECCD9CCE4CCEFCCFACD05CD1016
:10310C00CD1BCD26CD31CD3CCD47CD52CD5DCD683F
:10311C00CD73CD7FCD8ACD95CDA0CDABCDB6CDC168
:10312C00CDCCCDD7CDE2CDEDCDF8CE03CE0ECE1994
:10313C00CE24CE2FCE3ACE45CE50CE5BCE66CE71BF
:10314C00CE7CCE87CE92CE9DCEA8CEB3CEBECEC9EF
:10315C00CED4CEE0CEEBCEF6CF01CF0CCF17CF2214
:10316C00CF2DCF38CF43CF4ECF59CF64CF6FCF7A3F
:10317C00CF85CF90CF9BCFA6CFB1CFBCCFC7CFD26F
:10318C00CFDDCFE8CFF3CFFED009D014D01FD02A9B
:10319C00D035D040D04CD057D062D06DD078D083C1
:1031AC00D08ED099D0A4D0AFD0BAD0C5D0D0D0DBEF
:1031BC00D0E6D0F1D0FCD107D112D11DD128D1331A
:1031CC00D13ED149D154D15FD16AD175D180D18B47
:1031DC00D196D1A1D1ACD1B8D1C3D1CED1D9D1E472
:1031EC00D1EFD1FAD205D210D21BD226D231D23C99
:1031FC00D247D252D25DD268D273D27ED289D294C7
:10320C00D29FD2AAD2B5D2C0D2CBD2D6D2E1D2ECF6
:10321C00D2F7D302D30DD319D324D32FD33AD3451A
:10322C00D350D35BD366D371D37CD387D392D39D46
:10323C00D3A8D3B3D3BED3C9D3D4D3DFD3EAD3F576
:10324C00D400D40BD416D421D42CD437D442D44D9E
:10325C00D458D463D46ED479D485D490D49BD4A6CA
:10326C00D4B1D4BCD4C7D4D2D4DDD4E8D4F3D4FEF6
:10327C00D509D514D51FD52AD535D540D54BD5561E
:10328C00D561D56CD577D582D58DD598D5A3D5AE4E
:10329C00D5B9D5C4D5CFD5DAD5E6D5F1D5FCD60779
:1032AC00D612D61DD628D633D63ED649D654D65F9E
:1032BC00D66AD675D680D68BD696D6A1D6ACD6B7CE
:1032CC00D6C2D6CDD6D8D6E3D6EED6F9D704D70FFC
:1032DC00D71AD725D730D73BD746D752D75DD76823
:1032EC00D773D77ED789D794D79FD7AAD7B5D7C04E
:1032FC00D7CBD7D6D7E1D7ECD7F7D802D80DD8187B
:10330C00D823D82ED839D844D84FD85AD865D870A5
:10331C00D87BD886D891D89CD8A7D8B3D8BED8C9D2
:10332C00D8D4D8DFD8EAD8F5D900D90BD916D921F9
:10333C00D92CD937D942D94DD958D963D96ED97925
:10334C00D984D98FD99AD9A5D9B0D9BBD9C6D9D155
:10335C00D9DCD9E7D9F2D9FDDA08DA13DA1FDA2A7F
:10336C00DA35DA40DA4BDA56DA61DA6CDA77DA82A5
:10337C00DA8DDA98DAA3DAAEDAB9DAC4DACFDADAD5
:10338C00DAE5DAF0DAFBDB06DB11DB1CDB27DB3200
:10339C00DB3DDB48DB53DB5EDB69DB74DB7FDB8B2C
:1033AC00DB96DBA1DBACDBB7DBC2DBCDDBD8DBE355
:1033BC00DBEEDBF9DC04DC0FDC1ADC25DC30DC3B7F
:1033CC00DC46DC51DC5CDC67DC72DC7DDC88DC93AD
:1033DC00DC9EDCA9DCB4DCBFDCCADCD5DCE0DCECDC
:1033EC00DCF7DD02DD0DDD18DD23DD2EDD39DD44FE
:1033FC00DD4FDD5ADD65DD70DD7BDD86DD91DD9C2D
:10340C00DDA7DDB2DDBDDDC8DDD3DDDEDDE9DDF45C
:10341C00DDFFDE0ADE15DE20DE2BDE36DE41DE4C85
:10342C00DE58DE63DE6EDE79DE84DE8FDE9ADEA5AC
:10343C00DEB0DEBBDEC6DED1DEDCDEE7DEF2DEFDDC
:10344C00DF08DF13DF1EDF29DF34DF3FDF4ADF5504
:10345C00DF60DF6BDF76DF81DF8CDF97DFA2DFAD34
:10346C00DFB9DFC4DFCFDFDADFE5DFF0DFFBE0065B
:10347C00E011E01CE027E032E03DE048E053E05E84
:10348C00E069E074E07FE08AE095E0A0E0ABE0B6B4
:10349C00E0C1E0CCE0D7E0E2E0EDE0F8E103E10EE2
:1034AC00E119E125E130E13BE146E151E15CE16705
:1034BC00E172E17DE188E193E19EE1A9E1B4E1BF34
:1034CC00E1CAE1D5E1E0E1EBE1F6E201E20CE21761
:1034DC00E222E22DE238E243E24EE259E264E26F8C
:1034EC00E27AE286E291E29CE2A7E2B2E2BDE2C8B5
:1034FC00E2D3E2DEE2E9E2F4E2FFE30AE315E320E1
:10350C00E32BE336E341E34CE357E362E36DE3780B
:10351C00E383E38EE399E3A4E3AFE3BAE3C5E3D03B
:10352C00E3DBE3E6E3F2E3FDE408E413E41EE42961
:10353C00E434E43FE44AE455E460E46BE476E4818B
:10354C00E48CE497E4A2E4ADE4B8E4C3E4CEE4D9BB
:10355C00E4E4E4EFE4FAE505E510E51BE526E531E6
:10356C00E53CE547E552E55EE569E574E57FE58A0E
:10357C00E595E5A0E5ABE5B6E5C1E5CCE5D7E5E23B
:10358C00E5EDE5F8E603E60EE619E624E62FE63A65
:10359C00E645E650E65BE666E671E67CE687E69293
:1035AC00E69DE6A8E6B3E6BFE6CAE6D5E6E0E6EBBE
:1035BC00E6F6E701E70CE717E722E72DE738E743E4
:1035CC00E74EE759E764E76FE77AE785E790E79B13
:1035DC00E7A6E7B1E7BCE7C7E7D2E7DDE7E8E7F343
:1035EC00E7FEE809E814E81FE82BE836E841E84C68
:1035FC00E857E862E86DE878E883E88EE899E8A493
:10360C00E8AFE8BAE8C5E8D0E8DBE8E6E8F1E8FCC2
:10361C00E907E912E91DE928E933E93EE949E954EA
:10362C00E95FE96AE975E980E98CE997E9A2E9AD16
:10363C00E9B8E9C3E9CEE9D9E9E4E9EFE9FAEA0541
:10364C00EA10EA1BEA26EA31EA3CEA47EA52EA5D6A
:10365C00EA68EA73EA7EEA89EA94EA9FEAAAEAB59A
:10366C00EAC0EACBEAD6EAE1EAECEAF8EB03EB0EC5
:10367C00EB19EB24EB2FEB3AEB45EB50EB5BEB66EA
:10368C00EB71EB7CEB87EB92EB9DEBA8EBB3EBBE1A
:10369C00EBC9EBD4EBDFEBEAEBF5EC00EC0BEC1647
:1036AC00EC21EC2CEC37EC42EC4DEC59EC64EC6F6F
:1036BC00EC7AEC85EC90EC9BECA6ECB1ECBCECC79A
:1036CC00ECD2ECDDECE8ECF3ECFEED09ED14ED1FC7
:1036DC00ED2AED35ED40ED4BED56ED61ED6CED77F2
:1036EC00ED82ED8DED98EDA3EDAEEDB9EDC5EDD020
:1036FC00EDDBEDE6EDF1EDFCEE07EE12EE1DEE2846
:10370C00EE33EE3EEE49EE54EE5FEE6AEE75EE8071
:10371C00EE8BEE96EEA1EEACEEB7EEC2EECDEED8A1
:10372C00EEE3EEEEEEF9EF04EF0FEF1AEF25EF31CB
:10373C00EF3CEF47EF52EF5DEF68EF73EF7EEF89F1
:10374C00EF94EF9FEFAAEFB5EFC0EFCBEFD6EFE121
:10375C00EFECEFF7F002F00DF018F023F02EF0394B
:10376C00F044F04FF05AF065F070F07BF086F09278
:10377C00F09DF0A8F0B3F0BEF0C9F0D4F0DFF0EAA1
:10378C00F0F5F100F10BF116F121F12CF137F142CA
:10379C00F14DF158F163F16EF179F184F18FF19AF9
:1037AC00F1A5F1B0F1BBF1C6F1D1F1DCF1E7F1F229
:1037BC00F1FEF209F214F21FF22AF235F240F24B4A
:1037CC00F256F261F26CF277F282F28DF298F2A379
:1037DC00F2AEF2B9F2C4F2CFF2DAF2E5F2F0F2FBA9
:1037EC00F306F311F31CF327F332F33DF348F353D1
:1037FC00F35FF36AF375F380F38BF396F3A1F3ACF9
:10380C00F3B7F3C2F3CDF3D8F3E3F3EEF3F9F40427
:10381C00F40FF41AF425F430F43BF446F451F45C50
:10382C00F467F472F47DF488F493F49EF4A9F4B480
:10383C00F4BFF4CBF4D6F4E1F4ECF4F7F502F50DA7
:10384C00F518F523F52EF539F544F54FF55AF565D0
:10385C00F570F57BF586F591F59CF5A7F5B2F5BD00
:10386C00F5C8F5D3F5DEF5E9F5F4F5FFF60AF6152E
:10387C00F620F62BF637F642F64DF658F663F66E52
:10388C00F679F684F68FF69AF6A5F6B0F6BBF6C680
:10389C00F6D1F6DCF6E7F6F2F6FDF708F713F71EAD
:1038AC00F729F734F73FF74AF755F760F76BF776D8
:1038BC00F781F78CF798F7A3F7AEF7B9F7C4F7CF02
:1038CC00F7DAF7E5F7F0F7FBF806F811F81CF8272C
:1038DC00F832F83DF848F853F85EF869F874F87F58
:1038EC00F88AF895F8A0F8ABF8B6F8C1F8CCF8D788
:1038FC00F8E2F8EDF8F8F904F90FF91AF925F930AE
:10390C00F93BF946F951F95CF967F972F97DF988D7
:10391C00F993F99EF9A9F9B4F9BFF9CAF9D5F9E007
:10392C00F9EBF9F6FA01FA0CFA17FA22FA2DFA3831
:10393C00FA43FA4EFA59FA65FA70FA7BFA86FA915A
:10394C00FA9CFAA7FAB2FABDFAC8FAD3FADEFAE987
:10395C00FAF4FAFFFB0AFB15FB20FB2BFB36FB41B1
:10396C00FB4CFB57FB62FB6DFB78FB83FB8EFB99DF
:10397C00FBA4FBAFFBBAFBC5FBD1FBDCFBE7FBF20B
:10398C00FBFDFC08FC13FC1EFC29FC34FC3FFC4A30
:10399C00FC55FC60FC6BFC76FC81FC8CFC97FCA25F
:1039AC00FCADFCB8FCC3FCCEFCD9FCE4FCEFFCFA8F
:1039BC00FD05FD10FD1BFD26FD32FD3DFD48FD53B3
:1039CC00FD5EFD69FD74FD7FFD8AFD95FDA0FDABDF
:1039DC00FDB6FDC1FDCCFDD7FDE2FDEDFDF8FE030E
:1039EC00FE0EFE19FE24FE2FFE3AFE45FE50FE5B37
:1039FC00FE66FE71FE7CFE87FE92FE9EFEA9FEB464
:103A0C00FEBFFECAFED5FEE0FEEBFEF6FF01FF0C8C
:103A1C00FF17FF22FF2DFF38FF43FF4EFF59FF64B6
:103A2C00FF6FFF7AFF85FF90FF9BFFA6FFB1FFBCE6
:103A3C00FFC7FFD2FFDDFFE8FFF3FFFE303132336B
:073A4C003435363704020196
:100C9A0041004800C10441004900680000640000A6
:100CAA000001000100020002000300040004000524
:100CBA0000050006000600070008000800090009F0
:100CCA00000A000B000B000C000C000D000D000EBA
:100CDA00000F000F00100010001100120012001384
:100CEA00001300140015001500160016001700174F
:100CFA00001800190019001A001A001B001C001C19
:100D0A00001D001D001E001E001F002000200021E3
:100D1A0000210022002300230024002400250026AD
:100D2A00002600270027002800280029002A002A78
:100D3A00002B002B002C002D002D002E002E002F42
:100D4A00002F00300031003100320032003300340D
:100D5A0000340035003500360036003700380038D8
:100D6A0000390039003A003B003B003C003C003DA2
:100D7A00003E003E003F003F00400040004100426C
:100D8A000042004300430044004500450046004637
:100D9A0000470047004800490049004A004A004B02
:100DAA00004C004C004D004D004E004F004F0050CB
:100DBA000050005100510052005300530054005497
:100DCA000055005600560057005700580058005961
:100DDA00005A005A005B005B005C005D005D005E2B
:100DEA00005E005F006000600061006100620062F6
:100DFA0000630064006400650065006600670067C0
:100E0A000068006800690069006A006B006B006C8A
:100E1A00006C006D006E006E006F006F0070007154
:100E2A00007100720072007300730074007500751F
:100E3A000076007600770078007800790079007AE9
:100E4A00007A007B007C007C007D007D007E007FB4
:100E5A00007F00800080008100810082008300837F
:100E6A000084008400850086008600870087008849
:100E7A0000890089008A008A008B008B008C008D13
:100E8A00008D008E008E008F0090009000910091DE
:100E9A0000920092009300940094009500950096A9
:100EAA0000970097009800980099009A009A009B72
:100EBA00009B009C009C009D009E009E009F009F3E
:100ECA0000A000A100A100A200A200A300A300A408
:100EDA0000A500A500A600A600A700A800A800A9D2
:100EEA0000A900AA00AB00AB00AC00AC00AD00AD9D
:100EFA0000AE00AF00AF00B000B000B100B200B267
:100F0A0000B300B300B400B400B500B600B600B731
:100F1A0000B700B800B900B900BA00BA00BB00BCFB
:100F2A0000BC00BD00BD00BE00BE00BF00C000C0C6
:100F3A0000C100C100C200C300C300C400C400C590
:100F4A0000C500C600C700C700C800C800C900CA5B
:100F5A0000CA00CB00CB00CC00CC00CD00CE00CE26
:100F6A0000CF00CF00D000D100D100D200D200D3F0
:100F7A0000D400D400D500D500D600D600D700D8BA
:100F8A0000D800D900D900DA00DB00DB00DC00DC85
:100F9A0000DD00DD00DE00DF00DF00E000E000E150
:100FAA0000E200E200E300E300E400E500E500E619
:100FBA0000E600E700E700E800E900E900EA00EAE5
:100FCA0000EB00EC00EC00ED00ED00EE00EE00EFAF
:100FDA0000F000F000F100F100F200F300F300F479
:100FEA0000F400F500F600F600F700F700F800F844
:100FFA0000F900FA00FA00FB00FB00FC00FD00FD0E
:10100A0000FE00FE00FF00FF0100010101010102D4
:10101A00010201030104010401050105010601079A
:10102A0001070108010801090109010A010B010B65
:10103A00010C010C010D010E010E010F010F01102F
:10104A0001100111011201120113011301140115FA
:10105A0001150116011601170117011801190119C5
:10106A00011A011A011B011C011C011D011D011E8F
:10107A00011F011F01200120012101210122012359
:10108A000123012401240125012601260127012724
:10109A00012801280129012A012A012B012B012CEF
:1010AA00012D012E013001310132013301340135A4
:1010BA00013701380139013A013B013C013E013F48
:1010CA0001400141014201430145014601470148EE
:1010DA000149014A014C014D014E014F0150015293
:1010EA00015301540155015601570159015A015B37
:1010FA00015C015D015E01600161016201630164DD
:10110A000165016701680169016A016B016C016E81
:10111A00016F017001710172017301750176017726
:10112A0001780179017B017C017D017E017F0180CB
:10113A000182018301840185018601870189018A6F
:10114A00018B018C018D018E019001910192019315
:10115A0001940195019701980199019A019B019DBA
:10116A00019E019F01A001A101A201A401A501A65E
:10117A0001A701A801A901AB01AC01AD01AE01AF04
:10118A0001B001B201B301B401B501B601B701B9A9
:10119A0001BA01BB01BC01BD01BE01C001C101C24E
:1011AA0001C301C401C601C701C801C901CA01CBF3
:1011BA0001CD01CE01CF01D001D101D201D401D597
:1011CA0001D601D701D801D901DB01DC01DD01DE3D
:1011DA0001DF01E001E201E301E401E501E601E8E2
:1011EA0001E901EA01EB01EC01ED01EF01F001F186
:1011FA0001F201F301F401F601F701F801F901FA2C
:10120A0001FB01FD01FE01FF0200020102020204CC
:10121A0002050206020702080209020B020C020D6D
:10122A00020E020F02110212021302140215021612
:10123A0002180219021A021B021C021D021F0220B6
:10124A00022102220223022402260227022802295C
:10125A00022A022B022D022E022F02300231023301
:10126A0002340235023602370238023A023B023CA5
:10127A00023D023E023F024102420243024402454B
:10128A00024602480249024A024B024C024D024FF0
:10129A000250025102520253025402560257025A93
:1012AA00025C025F0261026302660268026A026D00
:1012BA00026F0272027402760279027B027D028058
:1012CA000282028402870289028B028E02900292B3
:1012DA00029502970299029C029E02A102A302A50C
:1012EA0002A802AA02AC02AF02B102B302B602B865
:1012FA0002BA02BD02BF02C102C402C602C902CBBF
:10130A0002CD02D002D202D402D702D902DB02DE17
:10131A0002E002E202E502E702E902EC02EE02F171
:10132A0002F302F502F802FA02FC02FF03010303C8
:10133A0003060308030A030D030F0311031403161C
:10134A000318031B031D0320032203240327032975
:10135A00032B032E03300332033503370339033CCF
:10136A00033E0340034303450348034A034C034F28
:10137A000351035303560358035A035D035F036182
:10138A00036403660368036B036D036F03720374DC
:10139A0003770379037B037E038003820385038734
:1013AA00038C03900395039A039F03A303A803AD39
:1013BA0003B103B603BB03BF03C403C903CE03D2FD
:1013CA0003D703DC03E003E503EA03EE03F303F8C0
:1013DA0003FD04010406040B040F04140419041E7B
:1013EA0004220427042C04300435043A043E04433E
:1013FA000448044D04510456045B045F0464046900
:10140A00046D04720477047C04800485048A048EC3
:10141A0004930498049C04A104A604AB04AF04B486
:10142A0004BD04C704D004DA04E304EC04F604FFA0
:10143A0005090512051B0525052E05380541054B2D
:10144A000554055D05670570057A0583058C0596C3
:10145A00059F05A905B205BB05C505CE05D805E159
:10146A000734088609D90B2B0C7E0DD00F23107573
:10147A0011C8131A146D15C01712186519B71B0A6B
:10148A001C5C1DAF1F01205421A722F9244C259E64
:10149A0026F1284329962AE82C3B2D8D2EE0410877
:1014AA00640041086500420866000041086800417E
:1014BA00000000410001014108690041086A004139
:1014CA00086B0042000200004200040000420006CD
:1014DA000000420008000042000A000042000C001E
:1014EA000041086C0041086D8041086E8042086F17
:1014FA000000410871004108728041087380420867
:03150A007400006A
:105B3C00900D02E0FEA3E0FF900CFEE0FCA3E0FD64
:105B4C00B50719ECB50615900D00E0FEA3E0FFEDCE
:0E5B5C00B50709ECB5060520C502D322C32209
:1019F000E4F584758810758902758E02758A017503
:061A00008C0143A8022244
:035D4400025A30D0
:0D5CFF00E4F584759A4075F809759D302212
:105C0500E4F58475E880900864E0F5BB7584027559
:105C1500BCF975E880A3E0F5BBE4F58443E71222FF
:075D2D00E4F58475D10222A8
:105C7F0075840F75A4CF75AD0175A50175A67F75D8
:095C8F00A77F75E10375E34022D3
:10590D00E4FFFE75840F438A0353A1DFF58475B759
:10591D003075840F43A120438901758D01758F0169
:10592D00758E040FBF00010EEF640F4E70F54389A5
:10593D0002E58920E4130FBF00010EBE0FF3BFFF78
:0C594D00F0E4F58443EF1080E875970249
:01595900222B
:101A1B0012590D125C7F1219F0125CFF125D2D1220
:051A2B005C05025D44B2
:104E710075FFDE75FFAD9000477453F0121A1BD217
:104E8100AF125C9802500FAF84E4F584900C78E087
:104E910004F08F84900049E06008121A33E4900016
:104EA10049F0125B0CEF60DF900D44E0FFB40B02A0
:104EB100D204EF64317044900047E0FF900D45E06B
:104EC1006F7038125B3C50FB900047E0FF125CDCD6
:104ED100125B3C50FB900D46E0FFA3E0FDA3E0FB1D
:104EE100A3E0900C7CF012502D125B3C50FB900023
:104EF10047E0FF125CC7125B3C50FB900D44E0643D
:104F010032703E900047E0FF900D45E06F70321225
:104F11005B3C50FB900047E0FF125CDC125B3C50B5
:104F2100FB900D46E0FFA3E0FDA3E0FB12189012F9
:104F31005B3C50FB900047E0FF125CC7125B3C50AA
:104F4100FB900D44E0642D703E900047E0FF900D12
:104F510045E06F7032125B3C50FB900047E0FF125E
:104F61005CDC125B3C50FB900D46E0FFA3E0FDA32F
:104F7100E0FB125495125B3C50FB900047E0FF129E
:104F81005CC7125B3C50FB900D44E0642E703E9078
:104F91000047E0FF900D45E06F7032125B3C50FB23
:104FA100900047E0FF125CDC125B3C50FB900D4629
:104FB100E0FFA3E0FDA3E0FB1253C2125B3C50FBF8
:104FC100900047E0FF125CC7125B3C50FB900D4420
:104FD100E0FFB414089000487401F0C205EFB41565
:104FE10005E4900048F0900048E07003024E88907C
:104FF1000D44E014601E046003024E88900D45E0EC
:10500100FFC3941E4003024E88900D1AEFF0125B0D
:10501100E3024E88900D45E0FFC3941E4003024E0B
:0C50210088900D1AEFF0121A33024E882E
:031A0600023A534E
:103A5300C0E0C0F0C083C082C0D075D000C000C039
:0D3A630001C002C003C004C005C006C007BA
:103A7000900CAE740FF0A374FFF0A37408F0A3745D
:103A800020F0900868E014600F146011146039246D
:103A9000037038125D408033125D0C802E900866F2
:103AA000E4F0A3F0124A35900867E004F070069045
:103AB0000866E004F0C3900867E09408900866E0A8
:103AC0006480948040DE8003125CB1900868E0045A
:103AD000F0C3648094844002E4F0900CB0E0FEA354
:103AE000E0FBAA06E4F9F8900CAEE0FEA3E0FFE4E8
:103AF000FCFD12439E900CAA1244E2900868E0FF7D
:0E3B000075F002124320AFF0EF700302420F87
:073B0E00900CB4E4F0A3F0F9
:103B1500900CB5E025E0FF900CB4E033FE743C2F2B
:103B2500F9741A3EFA900CD274FFF0A3EAF0A3E9F7
:103B3500F0900CD2E0FBA3E0FAA3E0F9124342FDBA
:103B4500540FFB900CD5E4F0A3EBF0EDC4540FFD3E
:103B5500A3E4F0A3EDF0900CD2E0FB90000112433A
:103B65005B540FFD900CD9E4F0A3EDF0741B2FF519
:103B750082740D3EF583E0FEA3E0FFE4FCFD900CAE
:103B8500DB1244E2900CB4E0FEA3E0FF4E6006EFCA
:103B950064054E7016900CD6E025E0FF900CD5E03C
:103BA50033FE74272FF58274008014900CB5E02540
:103BB500E0FF900CB4E033FE74252FF582740D3EC2
:103BC500F583E0FEA3E0FFE4FCFD900CCA1244E29D
:103BD500900CCAE0F8A3E0F9A3E0FAA3E0FBC374F4
:103BE500FF9BFF740F9AFEE499FDE498FCA3124431
:103BF500E2900CDBE0FCA3E0FDA3E0FEA3E0FFE424
:103C0500FBFAF9F8D31244D15069E47FAA7E02FD8C
:103C1500FC900CDBE0F8A3E0F9A3E0FAA3E0FBC31A
:103C25001244D1504E7F607EF07DFF7CFF900CDB0F
:103C3500E0F8A3A3A3E012439E900CBA1244E290CD
:103C45000CBAE0FCA3E0FDA3E0FEA3E0FFE47BAA41
:103C55007A02F9F81259EC900CBA1244E2900CBAB7
:103C6500E0FCA3E0FDA3E0FEA3E02428FFEE34235F
:103C7500023CF8900CDBE0FCA3E0FDA3E0FEA3E032
:103C8500FFE47BAA7A02F9F8D31244D15072E4FF1B
:103C95007E10FDFC900CDBE0F8A3E0F9A3E0FAA3AD
:103CA500E0FBC31244D150587F787EEC7DFF7CFF4A
:103CB500900CDBE0F8A3A3A3E012439E900CBA128C
:103CC50044E2900CBAE0FCA3E0FDA3E0FEA3E0FF14
:103CD500E47B567A0DF9F81259EC900CBA1244E2CD
:103CE500900CBAE0FCA3E0FDA3E0FEA3E0246FFF87
:103CF500EE3417FEE43DFDE43CFC900CBA1244E2C0
:103D0500900CBAE0FCA3E0FDA3E0FEA3E0FF900C5D
:103D1500C21244E2900CBAE0FCA3E0FDA3E0FEA3CE
:103D2500E0FF900CC61244E2900CCAE0FCA3E0FD53
:103D3500A3E0FEA3E0FF900CB61244E2900CB6E0BF
:103D4500FCA3E0FDA3E0FEA3E0FFE4FBFAF9F8D352
:103D55001244BB504DE4FF7E08FDFC900CB6E0F824
:103D6500A3E0F9A3E0FAA3E0FBC31244BB5033E49C
:103D75007FF47E01FDFC900CB6E0F8A3A3A3E0124E
:103D8500439E900CBA1244E2900CBAE0FCA3E0FD0D
:103D9500A3E0FEA3E0FFE4FB7A08F9F81259EC0270
:103DA5003EB7900CB6E0FCA3E0FDA3E0FEA3E0FF68
:103DB500E4FB7A08F9F8D31244BB506FE4FF7E0C9C
:103DC500FDFC900CB6E0F8A3E0F9A3E0FAA3E0FB54
:103DD500C31244BB5055E47FDC7E05FDFC900CB658
:103DE500E0F8A3A3A3E012439E900CBA1244E2901C
:103DF5000CBAE0FCA3E0FDA3E0FEA3E0FFE4FB7A40
:103E050004F9F81259EC900CBA1244E2900CBAE09D
:103E1500FCA3E0FDA3E0FEA3E0243CFFEE34F6FEA8
:103E2500ED34FFFDEC34FFFC023EB7900CB6E0FC30
:103E3500A3E0FDA3E0FEA3E0FFE4FB7A0CF9F8D3D1
:103E45001244BB5073E4FF7E10FDFC900CB6E0F805
:103E5500A3E0F9A3E0FAA3E0FBC31244BB5059E485
:103E65007F587E1BFDFC900CB6E0F8A3A3A3E012DF
:103E7500439E900CBA1244E2900CBAE0FCA3E0FD1C
:103E8500A3E0FEA3E0FFE47BFF7A03F9F81259EC07
:103E9500900CBA1244E2900CBAE0FCA3E0FDA3E05A
:103EA500FEA3E024B3FFEE34B5FEED34FFFDEC34A4
:103EB500FFFC900CBA1244E2900CC2E0F8A3E0F9C2
:103EC500A3E0FAA3E0FB900CBAE0FCA3E0FDA3E0BD
:103ED500FEA3E0FFEB2FFFEA3EFEE93DFDE83CFCDB
:103EE500900CC21244E2900CCEE0FCA3E0FDA3E0EE
:103EF500FEA3E0FF900CB61244E2900CB6E0FCA3E2
:103F0500E0FDA3E0FEA3E0FFE4FBFAF9F8D31244D9
:103F1500BB504DE4FF7E08FDFC900CB6E0F8A3E035
:103F2500F9A3E0FAA3E0FBC31244BB5033E47FF4EA
:103F35007E01FDFC900CB6E0F8A3A3A3E012439E1E
:103F4500900CBA1244E2900CBAE0FCA3E0FDA3E0A9
:103F5500FEA3E0FFE4FB7A08F9F81259EC0240757C
:103F6500900CB6E0FCA3E0FDA3E0FEA3E0FFE4FBBC
:103F75007A08F9F8D31244BB506FE4FF7E0CFDFCC0
:103F8500900CB6E0F8A3E0F9A3E0FAA3E0FBC312B6
:103F950044BB5055E47FDC7E05FDFC900CB6E0F893
:103FA500A3A3A3E012439E900CBA1244E2900CBA6C
:103FB500E0FCA3E0FDA3E0FEA3E0FFE4FB7A04F947
:103FC500F81259EC900CBA1244E2900CBAE0FCA33A
:103FD500E0FDA3E0FEA3E0243CFFEE34F6FEED3465
:103FE500FFFDEC34FFFC024075900CB6E0FCA3E04D
:103FF500FDA3E0FEA3E0FFE4FB7A0CF9F8D312443D
:10400500BB5073E4FF7E10FDFC900CB6E0F8A3E016
:10401500F9A3E0FAA3E0FBC31244BB5059E47F586F
:104025007E1BFDFC900CB6E0F8A3A3A3E012439E13
:10403500900CBA1244E2900CBAE0FCA3E0FDA3E0B8
:10404500FEA3E0FFE47BFF7A03F9F81259EC900C2C
:10405500BA1244E2900CBAE0FCA3E0FDA3E0FEA393
:10406500E024B3FFEE34B5FEED34FFFDEC34FFFC88
:10407500900CBA1244E2900CC6E0F8A3E0F9A3E074
:10408500FAA3E0FB900CBAE0FCA3E0FDA3E0FEA3DD
:10409500E0FFEB2FFFEA3EFEE93DFDE83CFC900C1E
:1040A500C61244E2E47F167E03FDFC900CC2E0F8E4
:1040B500A3E0F9A3E0FAA3E0FB12439E900CBE1225
:1040C50044E2900CBEE0FCA3E0FDA3E0FEA3E0FF0C
:1040D500E47B64FAF9F8124429900CBE1244E2E438
:1040E5007FFF7EFFFDFC900CBEE0F8A3E0F9A3E0A6
:1040F500FAA3E0FBD31244D1400A900CBE1244EE61
:104105000000FFFF900CBEA3A3E0FEA3E0FDAC06FC
:10411500900CD8E025E0FF900CD7E033FE744C2FCF
:10412500F58274003EF583ECF0A3EDF0E47F167E96
:1041350003FDFC900CC6E0F8A3E0F9A3E0FAA3E0C8
:10414500FB12439E900CBE1244E2900CBEE0FCA311
:10415500E0FDA3E0FEA3E0FFE47B64FAF9F8124476
:1041650029900CBE1244E2E47FFF7EFFFDFC900C1B
:10417500BEE0F8A3E0F9A3E0FAA3E0FBD31244D133
:10418500400A900CBE1244EE0000FFFF900CBEA347
:10419500A3E0FEA3E0FDAC06900CDAE025E0FF907D
:1041A5000CD9E033FE744C2FF58274003EF583EC98
:0441B500F0A3EDF096
:1041B900900CB5E004F07006900CB4E004F0900C9B
:1041C900B4E07004A3E064066003023B1578B27C96
:1041D9000C7D017B017A0079607E007F021242FA30
:1041E90078607C007D017B017A0079627E007F0224
:1041F9001242FA78627C007D017B017A0C79B27EE9
:06420900007F021242FAE0
:10420F00D007D006D005D004D003D002D001D00003
:0B421F00D0D0D082D083D0F0D0E032AD
:045D400043E8102202
:095D0C00758402D2ECE4F5842256
:104A3500900866E0FEA3E0FFEE6003024B96EFB43C
:104A450008004003024B96904A53F8282873024AFF
:104A55006B024A97024AC3024AEF024B1A024B38CD
:104A6500024B56024B7478E07C0C7D017B017A0089
:104A7500795C7E007F021242FA78E27C0C7D017B34
:104A8500017A00794C7E007F021242FA903A480280
:104A95004B9078E07C0C7D017B017A00795E7E008D
:104AA5007F021242FA78E27C0C7D017B017A007963
:104AB5004E7E007F021242FA903A49024B9078E00E
:104AC5007C0C7D017B017A0079607E007F021242B9
:104AD500FA78E27C0C7D017B017A0079507E007FBB
:104AE500021242FA903A4A024B9078E07C0C7D0122
:104AF5007B017A0079627E007F021242FA78E27CBD
:104B05000C7D017B017A0079527E007F021242FA08
:104B1500903A4B8076E4900CE0F0A3F078E27C0CC0
:104B25007D017B017A007954FE7F021242FA903AA8
:104B35004C8058E4900CE0F0A3F078E27C0C7D0109
:104B45007B017A007956FE7F021242FA903A4D8037
:104B55003AE4900CE0F0A3F078E27C0C7D017B0157
:104B65007A007958FE7F021242FA903A4E801CE490
:104B7500900CE0F0A3F078E27C0C7D017B017A00DB
:104B8500795AFE7F021242FA903A4FE493900CDF75
:104B9500F0E4F584C2FA900000E0F59B30FFFDC219
:104BA500FFE4FFFE0FBF00010EEF64324E70F5907B
:104BB5000CDFE0F59B30FFFDC2FFE4FEFF0FBF00F9
:104BC500010EEF64324E70F5900CE0E0F59B30FF7E
:104BD500FDC2FFE4FEFF0FBF00010EEF64324E7011
:104BE500F5900CE1E0F59B30FFFDC2FFE4FEFF0F01
:104BF500BF00010EEF64324E70F5900000E0F59BAA
:104C050030FFFDC2FFE4FEFF0FBF00010EEF64326F
:104C15004E70F5900CDFE0F59B30FFFDC2FFE4FE22
:104C2500FF0FBF00010EEF64324E70F5900CE2E00D
:104C3500F59B30FFFDC2FFE4FEFF0FBF00010EEF45
:104C450064324E70F5900CE3E0F59B30FFFDC2FF3A
:104C5500E4FEFF0FBF00010EEF64324E70F5D2FA8D
:014C6500222C
:031A3000024C66FF
:104C6600C0E0C0F0C083C082C0D075D000C000C014
:0D4C760001C002C003C004C005C006C00795
:104C830053E8DFAFBFEFFEADBE7C00E42DFFEC3E8B
:104C9300900024F0A3EFF0900024E0FCA3E0FD904B
:104CA3000864E0FF3395E0FEEF25E0FFEE33FE748A
:104CB300272FF58274003EF583ECF0A3EDF0900806
:104CC30064E004F0C3648094885003024E50E4F01F
:104CD300900031E0FFA3E0900010CFF0A3EFF0903D
:104CE300002FE0FFA3E0900012CFF0A3EFF09000BD
:104CF3002DE0FFA3E0900014CFF0A3EFF090002B82
:104D0300E0FFA3E0900016CFF0A3EFF0900029E0BE
:104D1300FFA3E0900018CFF0A3EFF0900027E0FF8F
:104D2300A3E090001ACFF0A3EFF090003FE0FFA3C1
:104D3300E090001CCFF0A3EFF0900041E0FFA3E070
:104D430090001ECFF0A3EFF0900043E0FFA3E090AC
:104D53000020CFF0A3EFF0900045E0FFA3E0900028
:104D630022CFF0A3EFF0900001E06037E4FFEF25DE
:104D7300E02410F582E43400F583E0FCA3E0FDEFCA
:104D830025E0242FF582E4340DF583ECF0A3EDF058
:104D93000FEFB40AD9900001E004F0E0D3940F4080
:104DA30002E4F0900001E070047D0180027D007F49
:104DB30000121535900001E070047D0180027D0032
:104DC3007F01121535900001E070047D0180027DA2
:104DD300007F02121535900001E070047D0180020E
:104DE3007D007F03121535900001E070047D018082
:104DF300027D007F04121535900001E070047D01EF
:104E030080027D007F05121535900001E070047D5E
:104E13000180027D007F06121535900001E07004C9
:104E23007D0180027D007F07121535900001E0703F
:104E3300047D0180027D007F08121535900001E09A
:104E430070047D0180027D007F091215359008648E
:034E5300E0F5BBCC
:104E5600D007D006D005D004D003D002D001D000B0
:0B4E6600D0D0D082D083D0F0D0E0325A
:031A39000257DF72
:1057DF00C0E0C0F0C083C082C0D075D000C005C08B
:1057EF0006C007758402C2ED900026E5BEF0E07595
:1057FF00F010A4FD900865E0FF3395E0FEEF25E083
:10580F00FFEE33FE74372FF58274003EF583E5F01B
:10581F00F0A3EDF0900865E004F0C3648094884035
:10582F0002E4F0900865E0F5BB758400D007D00660
:0D583F00D005D0D0D082D083D0F0D0E032A0
:10555B00900039A3E0FEC394F040047F108016EE58
:10556B00C3944040047F20800CEED3942040047FF2
:10557B00408002E4FF90086AE033333354F8FEA313
:10558B00E0903A50934EFE900048E0C433333354CE
:06559B00804E4FFEC2909D
:1055A100900CDFE4F0A37410F0900CDF74FFF5F0C1
:0E55B100124388FCD3E5F09400EC940050EB1C
:1055BF00E4FDEEA805088002C313D8FC139286C23F
:0155CF008754
:1055D000900CDFE4F0A37410F0900CDF74FFF5F092
:0E55E000124388FAD3E5F09400EA940050EBF1
:0255EE00D28762
:1055F000900CDFE4F0A37410F0900CDF74FFF5F072
:0E560000124388FAD3E5F09400EA940050EBD0
:07560E000DEDB408AED290CF
:015615002272
:1045820090003BE0FFA3E0900002CFF0A3EFF09099
:10459200003DE0FEA3E0FF900004EEF0A3EFF0D3B5
:1045A200900007E09F900006E09E5016900004E005
:1045B200FFA3E0A3CFF0A3EFF090000AE4F0A3740E
:1045C20080F0900008E0FEA3E0FF900002E0FCA370
:1045D200E0FDC39FEC9E4011900008ECF0A3EDF0CB
:1045E20090000CE4F0A37480F0900004E0FEA3E0DD
:1045F200FFD394A3EE94004003D38001C392B0D3BF
:10460200EF94F4EE94004003D38001C392B1900082
:1046120004E0FEA3E0FFD3943BEE94024003D38078
:1046220001C392B2D3EF94D3EE94034003D380013B
:10463200C392B3900004E0FEA3E0FFD394BCEE94D7
:10464200054003D38001C392B4D3EF9433EE940AAE
:104652004003D38001C392B5D3900005E0944C90FF
:104662000004E0940F4003D38001C392B6D39000BC
:104672000BE0940090000AE094004070900006E085
:10468200FEA3E0FFD3944CEE940F4004D2B6804CCC
:10469200D3EF9433EE940A4004D2B5803FD3EF9423
:1046A200BCEE94054004D2B48032D3EF94D3EE949E
:1046B200034004D2B38025D3EF943BEE940240042E
:1046C200D2B28018D3EF94F4EE94004004D2B180B9
:1046D2000BD3EF94A3EE94004002D2B090000BE013
:1046E20024FFF090000AE034FFF08007E490000617
:1046F200F0A3F0D3ED94A3EC94004003D38001C364
:1047020092A0D3ED94F4EC94004003D38001C392C1
:10471200A1900002E0FEA3E0FFD3943BEE9402409E
:1047220003D38001C392A2D3EF94D3EE9403400348
:10473200D38001C392A3900002E0FEA3E0FFD394D2
:10474200BCEE94054003D38001C392A4D3EF94330B
:10475200EE940A4003D38001C392A5D3900003E0F4
:10476200944C900002E0940F4003D38001C392A6C0
:10477200D390000DE0940090000CE0940040709003
:104782000008E0FEA3E0FFD3944CEE940F4004D265
:10479200A6804CD3EF9433EE940A4004D2A5803F16
:1047A200D3EF94BCEE94054004D2A48032D3EF94AC
:1047B200D3EE94034004D2A38025D3EF943BEE942E
:1047C200024004D2A28018D3EF94F4EE9400400485
:1047D200D2A1800BD3EF94A3EE94004002D2A0901A
:1047E200000DE024FFF090000CE034FFF08007E4BD
:0947F200900008F0A3F012555BE1
:0147FB00229B
:0F1A090090086BE004F0E0D394024002E4F02276
:085D150090086AE06401F0222D
:1051DD0090086DE0A3F0E5B0548090086DF0A3E069
:1051ED00FD90086DE0FE6D90000EF0EE703FED60ED
:1051FD0007E490086FF0A3F0900870E004F07006DB
:10520D0090086FE004F0D3900870E094D090086F90
:10521D00E09400404D90086CE0700A900047E0FF6C
:10522D007D0D125C2590086C7401F0803590086E30
:10523D00E0702FC3900870E094D090086FE0940058
:10524D00501B300409900048E06401F0800F90007D
:10525D0048E06009A37401F0E4900048F0E4900880
:10526D006CF0900872E0A3F0E5A05480900872F005
:10527D00A3E0FD900872E0FE6D90000FF0EE703728
:10528D00ED6007E4900874F0A3F0900875E004F069
:10529D007006900874E004F0D3900875E094C09007
:1052AD000874E09400402D900871E07003125D15B4
:1052BD009008717401F022900873E07017C3900884
:1052CD0075E094C0900874E094005003121A09E43C
:0452DD00900871F0D4
:0152E10022AA
:105CB100900869E070051251DD8003124582900859
:065CC10069E06401F0221D
:06150D00410D1A00C105AA
:10575500125D25E4900C7BF0900C7BE0FFC3940672
:105765005018EF25E0241BF582E4340DF583E4F0B1
:10577500A3F0900C7BE004F080DE900C7B7406F0C7
:10578500900C7BE0FFC3940A501BEF25E0241BF52A
:1057950082E4340DF5837407F0A374FFF0900C7B5D
:1057A500E004F080DBE4900C7BF0900C7BE0FFC321
:1057B500941E502375F014EFA42401F582E5F0340E
:1057C50080AF82FE7C0D7D1B7B147A001259A6905A
:0A57D5000C7BE004F080D3025B9629
:105ADC00900C797402F0E4A3F0125D257E807F00B7
:105AEC007C0C7D797B017A001259A67E827F597CD1
:105AFC000C7D7A7B017A001259A6125B96025755DF
:105C450030040F20050C900048E06006125D1DD25F
:0E5C55000522200408900048E0700204F022AE
:105C9800908259E493600C908000E493640260035E
:095CA800125ADCE4900D1AF022FE
:105BE300900D1AE075F014A42401F9748035F0FACD
:105BF3007BFF781B7C0D7D017E007F141242FAC26D
:025C0300052278
:105BBF00125D25900D1AE075F014A42401F582E50D
:105BCF00F03480AF82FE7C0D7D1B7B147A0012595E
:045BDF00A6025B9629
:061A3300125BBFC2052298
:0A502D00900C7AEDF0900C79EFF092
:10503700D39B500302510BE024FFFEE434FF900C96
:105047007EF0A3CEF0EB14900C7DF0900C7AE02468
:10505700FFFFE434FFFE900C7EE0FCA3E0FDD39F4E
:10506700EE6480F8EC64809840030251DC90800184
:1050770075F014ED12451FEC75F014A42583AF826B
:10508700900C85F0A3EFF0900C7DE075F014A4244C
:1050970001F9748035F0FA900C8274FFF0A3EAF0FE
:1050A700A3E9F0E4900C80F0A3F0900C82A3E475E0
:1050B700F001124388FEAFF0900C85E475F0011201
:1050C700438885F082F583E493FD1256BF900C81E7
:1050D700E004F07006900C80E004F0C3900C81E0CF
:1050E7009414900C80E0940040C0125B96900C7F63
:1050F700E004F07006900C7EE004F0900C7DE00474
:10510700F0025052900C7AE024FFFEE434FF900C3A
:105117007EF0A3CEF0900C7CE014A3F0900C79E025
:1051270024FFFFE434FFFE900C7EE0FCA3E0FDC308
:105137009FEE6480F8EC64809850030251DC908005
:105147000175F014ED12451FEC75F014A42583AF1B
:1051570082900C85F0A3EFF0900C7DE075F014A41D
:105167002401F9748035F0FA900C8274FFF0A3EAF9
:10517700F0A3E9F0E4900C80F0A3F0900C82A3E494
:1051870075F001124388FEAFF0900C85E475F001CD
:1051970012438885F082F583E493FD1256BF900C85
:1051A70081E004F07006900C80E004F0C3900C815D
:1051B700E09414900C80E0940040C0125B96900C31
:1051C7007FE024FFF0900C7EE034FFF0900C7DE050
:0551D70014F002512359
:0151DC0022B0
:05189000900C79EDF061
:10189500EF14900C93F0EB14A3F0900C79E014FF87
:1018A500900C93E0D39F40030219EFA3E075F01469
:1018B500A42401F582E5F03480AF82FEE4900C9516
:1018C500F0A3F0900C95E0FCA3E0FDC39414EC9418
:1018D50000502B0FEFAA0670010E14F5828A83E4DF
:1018E50093FB747F2DF582E4340CF583EBF0900CBB
:1018F50096E004F070CD900C95E004F080C5900C56
:1019050094E075F014A42401F9748035F0FA900C74
:101915007A74FFF0A3EAF0A3E9F0900C93E075F078
:1019250014A42401F582E5F03480AF82900C7DF09B
:10193500A3EFF0E4900C95F0A3F0900C7AA3E47576
:10194500F001124388FEAFF0900C7DE475F00112B2
:10195500438885F082F583E493FD1256BF900C967B
:10196500E004F07006900C95E004F0C3900C96E04E
:101975009414900C95E0940040C0900C93E075F0A1
:1019850014A42401F9748035F0FA900C7A74FFF0F0
:10199500A3EAF0A3E9F0E4900C95F0A3F0900C9580
:1019A500E0FCA3E0FDC39414EC9400502D900C7A58
:1019B500A3E475F001124388FEAFF0747F2DF58224
:1019C500E4340CF583E0FD1256BF900C96E004F06C
:1019D50070CB900C95E004F080C3125B96900C934D
:0A19E500E004F0A3E004F002189FF4
:0119EF0022D5
:0753C200900C79EBF0AC0741
:1053C900A2AFE433A3F0AF05A3E4F0A3EFF0E07FCD
:1053D90000FE900C7BF0A3EFF0AD04EDFF900C7B89
:1053E900EEF0A3EFF0C2AF900D1A740FF0125D2525
:1053F900900D1AE075F014A42401F9748035F0FABF
:10540900900C7F74FFF0A3EAF0A3E9F0E4900C7D1F
:10541900F0A3F0900C7BE0FCA3E0FFECFD900C798D
:10542900E0FBE4900C86F0D2021252E2900C82EF7B
:10543900F0FD900C7FA3E475F001124388FEAFF0F4
:105449001256BF900C7CE004F07006900C7BE004CF
:10545900F0900C7EE004F07006900C7DE004F0C33F
:10546900900C7EE09414900C7DE0940040A5125BB2
:1054790096900D1AE004F0E0C3941E50030253F60F
:0B548900125A30900C7AE024FF92AF22
:0154940022F5
:07549500900C79EBF0AC076D
:10549C00A2AFE433A3F0AF05900C7DE4F0A3EFF0E2
:1054AC00E07F00FE900C7DF0A3EFF0AD04EDFF90DB
:1054BC000C7DEEF0A3EFF0C2AF900D1A740FF090CC
:1054CC000D1AE0FFC3941E507A75F014EFA424015A
:1054DC00F582E5F03480AF82900C7FF0A3EFF0E41E
:1054EC00900C7BF0A3F0900C7DE0FCA3E0FFECFDB6
:1054FC00900C79E0FB900C7FE475F00112438885E9
:10550C00F082F583E493900C86F0C2021252E29082
:10551C000C7EE004F07006900C7DE004F0900C7CA6
:10552C00E004F07006900C7BE004F0C3900C7CE07F
:10553C009414900C7BE0940040AC900D1AE004F0B5
:0E554C000254CB125A30900C7AE024FF92AF3A
:01555A00222E
:10151300540D2F0000000000000000000000000038
:0715230000000000000000C1
:1015350090FFFF124551EDF090FFFF124551EFF07E
:0615450090FFEE1245517B
:10154B00850883850982E4F0A3F09000121245759B
:10155B00E025E0242FF582E4340DF583E0FEA3E0D3
:10156B00FFFBAA06E4F9F8900012124575E025E09E
:10157B002410F582E43400F583E0FEA3E0FFC3EF13
:10158B009BFFEE9AFEE499FDE498FC8508838509A0
:10159B0082A3A31244E2E47F40FEFDFC8508838511
:1015AB000982A3A3E0F8A3E0F9A3E0FAA3E0FBC34D
:1015BB001244BB400B850883850982E4F0A304F039
:1015CB0074FF7FC0FEFDFC850883850982A3A3E021
:1015DB00F8A3E0F9A3E0FAA3E0FBD31244BB500B52
:1015EB0085088385098274FFF0A3F085088385093C
:1015FB0082E0FEA3E0FF4E700302188AEFF4700244
:07160B00EEF4600302171763
:10161200900012124575E025E0242FF582E4340D86
:10162200F583E0FEA3E0FFE4FCFD90000E12457599
:101632001244E2E47F01FEFDFC90000E124575E0CB
:10164200F8A3E0F9A3E0FAA3E0FBC31244BB500DF8
:1016520090000E1245751244EE0000000190001237
:10166200124575E025E0241BF582E4340DF583E094
:10167200FEA3E0FFE4FCFD7BFF7A0FF9F812439E24
:1016820090000E124575E0F8A3E0F9A3E0FAA3E09A
:10169200FB1259EC9000061245751244E2900012BA
:1016A200124575E025E02410F582E43400F583E06C
:1016B200FEA3E0FFE4FCFD900006124575E0F8A3EE
:1016C200E0F9A3E0FAA3E0FB12439E90000A124560
:1016D200751244E2E47BFF7A0FF9F890000A124592
:1016E20075E0FCA3E0FDA3E0FEA3E0FF1259EC903D
:1016F2000012124575E025E0241BF582E4340DF555
:1017020083EEF0A3EFF0900013124575E070030230
:0217120018615C
:1017140002185E850883850982E0FEA3E064014E19
:051724006003021861E2
:10172900900012124575E025E0241BF582E4340D82
:10173900F583E0FEA3E0FBC374FF9BFF740F9EFEDD
:10174900E49400FDE49400FCE47BFF7A0FF9F812BD
:10175900439E9000061245751244E290001212450C
:1017690075E025E0242FF582E4340DF583E0FEA32E
:10177900E0FBC374FF9BFF740F9EFEE49400FDE43D
:101789009400FC90000A1245751244E2E47F01FEC0
:10179900FDFC90000A124575E0F8A3E0F9A3E0FA10
:1017A900A3E0FBC31244BB500D90000A1245751209
:1017B90044EE00000001900006124575C083C08206
:1017C900E0FCA3E0FDA3E0FEA3E0FF90000A1245C0
:1017D90075E0F8A3E0F9A3E0FAA3E0FB1259ECD015
:1017E90082D0831244E2900012124575E025E0246C
:1017F90010F582E43400F583E0FEA3E0FBC374FF37
:101809009BFF740F9EFEE49400FDE49400FC90009D
:1018190006124575E0F8A3E0F9A3E0FAA3E0FB128C
:10182900439EE47BFF7A0FF9F81259ECC374FF9FCA
:10183900FF740F9EFE900012124575E025E0241BEF
:10184900F582E4340DF583EEF0A3EFF09000131266
:081859004575E06003125C45D7
:10186100900012124575E0FF25E02410F582E43462
:1018710000F583E0FCA3E0FDEF25E0242FF582E4F1
:09188100340DF583ECF0A3EDF049
:06188A009000140245511C
:105C2500900CDFEFF0A3EDF07F0A125616900CDF13
:105C3500E0FF125616900CE0E0FF125616025CF1DA
:085D1D007F02125616025CF130
:065B0C00125D34EF60277A
:105B1200900C79740DF0A37443F0125AA6900C798C
:105B2200E475F00112438885F082F583EFF0125D8F
:075B32003AEF70E67F01224B
:035B39007F0022C8
:105CC700900C79EFF07F2F125616900C79E0FF12A7
:055CD7005616025CF10D
:105CDC00900C79EFF07F30125616900C79E0FF1291
:055CEC005616025CF1F8
:0A152A00410D1800410D1900C10128
:105C6300AF84E4F584C2C343E60243F60275C3017D
:0B5C730075C04475CF8F43C3018F84C0
:015C7E002203
:105A30007E0C7FEA900CE8EEF0A3EFF0900CE6EE1F
:105A4000F0A3EFF0900CE4EEF0A3EFF07E0D7F04F6
:105A5000900D02EEF0A3EFF0900D00EEF0A3EFF04A
:0D5A6000900CFEEEF0A3EFF0C200025C63BC
:105A6D00900CE6E475F00112438885F082F583EF22
:105A7D00F0900CE6E475F00112438885F082F58311
:105A8D00EDF0900CE6E0B40C0FA3E0B4FE0A900C20
:095A9D00E6740CF0A374EAF02297
:0D5CF100AF84E4F584C200C2C4D2C58F8424
:015CFE002283
:10561600200055D200900D00E475F00112438885F4
:10562600F082F58374FFF07C0D7D18900D00E0B5D7
:10563600040FA3E0B5050A900D00740DF0A37404E1
:10564600F0900D00E475F00112438885F082F58331
:10565600E4F0900D00E0B5040FA3E0B5050A900D47
:1056660000740DF0A37404F0900D00E475F00112BF
:10567600438885F082F583E4F0900D00E0B40D0FC9
:10568600A3E0B4180A900D00740DF0A37404F09012
:105696000D00E475F00112438885F082F583EFF082
:1056A600900D00E0B40D0FA3E0B4180A900D00743D
:0956B6000DF0A37404F07F012241
:105B6A00900CE8E0FCA3E0FD900CE4E0B50408A387
:105B7A00E0B505037F0022900CE8E0FCA3E0F58283
:0C5B8A008C83E0B507037F01227F00221E
:105AA600900CE9E004F07006900CE8E004F0900C2D
:105AB600E8E475F00112438885F082F583E0FF90F3
:105AC6000CE8E0B40C0FA3E0B4FE0A900CE8740CEA
:055AD600F0A374EAF0EA
:015ADB0022A8
:065D34007FFF125B6A22F2
:065D3A00E4FF125B6A2287
:031A18000247FC86
:1047FC00C0E0C0F0C083C082C0D075D000C000C083
:10480C0004C005C006C007E5C154F812452B49F198
:10481C000048570848571048A51848F12048FE286A
:10482C0049893049953849A65049A65849B9604933
:10483C00A86849B97049A87849A68049C88849A68A
:10484C009049C89849D9A000004A1EC2C5900CFFD7
:10485C00E004F07006900CFEE004F07E0D7F1890E2
:10486C000CFEE0B5060FA3E0B5070A900CFE740D24
:10487C00F0A37404F0900CFEE475F00112438885EB
:10488C00F082F583E0F5C2900CFEE06E7003A3E0BD
:10489C006F6003024A1E02497C900CFFE004F0702A
:1048AC0006900CFEE004F07E0D7F18900CFEE0B537
:1048BC00060FA3E0B5070A900CFE740DF0A3740468
:1048CC00F0900CFEE475F00112438885F082F583BC
:1048DC00E0F5C2900CFEE06E7003A3E06F60030283
:1048EC004A1E02497C900D02E0FFA3E0900CFECF23
:1048FC00801B900D00E0FEA3E0FF900CFEE0FCA3FB
:10490C00E0FDB50713ECB5060F900D02EEF0A3EF2A
:10491C00F0C2C5D2C4024A1E8D828C83E0B4FF075C
:10492C00C2C4D2C5024A1E900CFFE004F07006907F
:10493C000CFEE004F07E0D7F18900CFEE0B5060F27
:10494C00A3E0B5070A900CFE740DF0A37404F0906C
:10495C000CFEE475F00112438885F082F583E0F5D6
:10496C00C2900CFEE06E7003A3E06F6003024A1E5F
:10497C00900CFE740DF0A37404F0024A1E900D020C
:10498C00E0FFA3E0900CFE803B900D02E0FFA3E063
:10499C00900CFECFF0A3EFF080788017900D02E022
:1049AC00FFA3E0900CFECFF0A3EFF0D201ADC27FDD
:1049BC00FF8004ADC2E4FF125A6D8056900CE4E007
:1049CC00FFA3E0A3CFF0A3EFF0D2C48045900CE698
:1049DC00E0FFA3E0900CE4CFF0A3EFF0300133D272
:1049EC00C5C201802D900D02E0FEA3E0FF900CFEED
:1049FC00EEF0A3EFF0900CE4E0FDA3E0A3CDF0A368
:104A0C00EDF0D2C4900D00E06E7003A3E06F600275
:104A1C00D2C5C2C3D007D006D005D004D000D0D0A8
:094A2C00D082D083D0F0D0E0323A
:10595A00900C9EE584F0A2AF9202AF01AE027C00E9
:10596A00E4FDA31244E2900CA1E0FEA3E0780AA6AB
:10597A000608F6E4F584C2AF43B701438F02438FAA
:10598A000118E6FE08E6F5828E83E4F053B7FEF5C9
:0B599A008FA20292AF900C9EE0F584FB
:0159A50022DF
:0558B100900CA4EDF0D5
:1058B600A3E584F0A2AF9202AF01AE027C00E4FD44
:1058C600A31244E2900CA4E0FFFD3395E0FCEDF456
:1058D6004C6029900CA8E0FCA3E0780AA60408F620
:1058E600E4F584C2AF43B701758F0118E6FC08E6FC
:1058F600F5828C83EFF053B7FEE4F58FA20292AFE8
:06590600900CA5E0F58401
:01590C002278
:10584C00900C9EEEF0A3EFF0A3ECF0A3EDF0A3EA26
:10585C00F0A3EBF0900CA2E07002A3E06046900C79
:10586C009EE0FEA3E0AA06F97B01A3E0FEA3E0F50F
:10587C00828E83E0FD1258B1900CA3E024FFF090CF
:10588C000CA2E034FFF0900CA1E004F07006900C38
:10589C00A0E004F0900C9FE004F070B8900C9EE037
:0558AC0004F080B022B1
:085D2500E4900C76F0A3F022DB
:105B9600900C76E0FEA3E0AA06F97B0112595A9012
:105BA6000C76E0FEA3E0FF7C087D761B7A04125893
:095BB6004CE4900C76F0A3F022FF
:0D56BF00900C99EDF0900C97EEF0A3EFF039
:1056CC00EE54FCFE900C76E0FCA3E0FD7002EE6C58
:1056DC006059ED4C6003125B96900C97E0FEEE5413
:1056EC00FCFE7F00900C76F0A3EFF0900C9AEEF09D
:1056FC00A3EFF0A37408F0A37476F07FFF7E039001
:10570C000C9AE475F00112438885F082F583E493DA
:10571C00FD900C9CE475F00112438885F082F583B2
:10572C00EDF0EF1F70011EEF4E70D4900C99E0FF5E
:10573C00900C97E0FCA3E0FDEC5403FC74762DF583
:08574C008274083CF583EFF0C4
:015754002232
:1059A600900C7CEEF0A3EFF0A3ECF0A3EDF0A3EAED
:1059B600F0A3EBF0900C8074FFF5F012438845F0ED
:1059C6006023900C7CE475F001124388AFF0FE90E2
:1059D6000C7EE475F00112438885F082F583E0FDC4
:0659E6001256BF80CF2223
:0752E200900C83EFF0A90519
:1052E900C20320C3FD20C5FAC2C4D2C5E4FFFD3004
:1052F900C3FD30C3FDE5C154F8FC64086004ECB497
:105309001013EFB40105EB44018003EB54FEF5C221
:105319007D010253B0ECB4180B89C27D02C2C4C22C
:10532900C50253B0ECB420028045EC6428703CED12
:10533900B4020E900C83E0F5C27D03C2C5C2C480DD
:1053490066EDB4031B300208D2C57F01C2C4805781
:10535900900C86E0F5C2C2C57D04E4FFC2C4804753
:10536900ED64047042D2C47D05803CECB4300AD2AD
:10537900C4D2C57D08E4FF802EECB438028024EC49
:10538900B44006C2C2C2C5801EECB448028014EC07
:10539900B450028004ECB4580AD2C47D07AEC2C22C
:1053A900C28004D2C4D2C5C2C3ED64076008ED64EB
:0853B9000560030252FBAF0680
:0153C10022C9
:100C1A00024E71E493A3F8E493A34003F68001F231
:100C2A0008DFF48029E493A3F85407240CC8C333DB
:100C3A00C4540F4420C8834004F456800146F6DFAA
:100C4A00E4800B0102040810204080900C9AE47E94
:100C5A00019360BCA3FF543F30E509541FFEE4939F
:100C6A00A360010ECF54C025E060A840B8E493A366
:100C7A00FAE493A3F8E493A3C8C582C8CAC583CA91
:100C8A00F0A3C8C582C8CAC583CADFE9DEE780BE49
:0115340000B6
:10422A00E709F608DFFA8046E709F208DFFA803E76
:10423A0088828C83E709F0A3DFFA8032E309F60863
:10424A00DFFA8078E309F208DFFA807088828C83CB
:10425A00E309F0A3DFFA806489828A83E0A3F6087F
:10426A00DFFA805889828A83E0A3F208DFFA804C59
:10427A0080D280FA80C680D4806980F28033801030
:10428A0080A680EA809A80A880DA80E280CA803399
:10429A0089828A83ECFAE493A3C8C582C8CCC58311
:1042AA00CCF0A3C8C582C8CCC583CCDFE9DEE780E1
:1042BA000D89828A83E493A3F608DFF9ECFAA9F060
:1042CA00EDFB2289828A83ECFAE0A3C8C582C8CCB6
:1042DA00C583CCF0A3C8C582C8CCC583CCDFEADECF
:1042EA00E880DB89828A83E493A3F208DFF980CC31
:1042FA0088F0EF60010E4E60C388F0ED2402B4042A
:10430A000050B9F582EB2402B4040050AF232345D0
:06431A00822390427A7339
:10432000C2D530F707B2D563F0FF05F030E70CB225
:10433000D5F4048463F0FF05F080018430D502F4E5
:02434000042255
:10434200BB010689828A83E0225002E722BBFE0279
:09435200E32289828A83E49322AC
:10435B00BB010CE58229F582E5833AF583E0225017
:10436B0006E92582F8E622BBFE06E92582F8E22261
:0D437B00E58229F582E5833AF583E493227B
:10438800A3F8E0C5F025F0F0E582158270021583E8
:06439800E0C838F0E82245
:10439E00E88FF0A4CC8BF0A42CFCE98EF0A42CFCBE
:1043AE008AF0EDA42CFCEA8EF0A4CDA8F08BF0A43C
:1043BE002DCC3825F0FDE98FF0A42CCD35F0FCEB9B
:1043CE008EF0A4FEA9F0EB8FF0A4CFC5F02ECD3960
:0F43DE00FEE43CFCEAA42DCE35F0FDE43CFC22CD
:1043ED0075F008758200EF2FFFEE33FECD33CDCC87
:1043FD0033CCC58233C5829BED9AEC99E58298400A
:10440D000CF582EE9BFEED9AFDEC99FC0FD5F0D6E6
:10441D00E4CEFBE4CDFAE4CCF9A88222B800C1B910
:10442D000059BA002DEC8BF084CFCECDFCE5F0CB4E
:10443D00F97818EF2FFFEE33FEED33FDEC33FCEB87
:10444D0033FB10D703994004EB99FB0FD8E5E4F942
:10445D00FA227818EF2FFFEE33FEED33FDEC33FC2F
:10446D00C933C910D7059BE99A4007EC9BFCE99A23
:10447D00F90FD8E0E4C9FAE4CCFB2275F010EF2F68
:10448D00FFEE33FEED33FDCC33CCC833C810D70768
:10449D009BEC9AE899400AED9BFDEC9AFCE899F8A3
:0E44AD000FD5F0DAE4CDFBE4CCFAE4C8F92236
:1059EC00C2D5E830E70FB2D5E4C39BFBE49AFAE4E6
:1059FC0099F9E498F8EC30E717B2D5125A22124410
:105A0C0029E4C39BFBE49AFAE499F9E498F880033F
:105A1C0012442930D50DE4C39FFFE49EFEE49DFDA6
:045A2C00E49CFC22D8
:1044BB00EB9FF5F0EA9E42F0E99D42F0EC6480C878
:0644CB0064809845F02218
:1044D100EB9FF5F0EA9E42F0E99D42F0E89C45F041
:0144E10022B8
:0C44E200ECF0A3EDF0A3EEF0A3EFF0224D
:1044EE00A8828583F0D083D082124505124505122D
:1044FE004505124505E473E493A3C583C5F0C58352
:10450E00C8C582C8F0A3C583C5F0C583C8C582C817
:01451E00227A
:0C451F00A42582F582E5F03583F58322A7
:10452B00D083D082F8E4937012740193700DA3A31F
:10453B0093F8740193F5828883E473740293686033
:06454B00EFA3A3A380DF33
:10455100E5092582F582E5083583F583B5080485EB
:1045610082092210AF06858209F50822858209F5A4
:0445710008D2AF229B
:0D457500E5092582F582E5083583F58322EE
:00000001FF
